:100000000C9483030C94AB030C94AB030C94AB03E0
:100010000C94AB030C94AB030C94AB030C94AB03A8
:100020000C94AB030C94AB030C94AB030C947D1FAA
:100030000C94AB030C94AB030C94AB030C94AB0388
:100040000C9462200C94AB030C94AB030C94AB03A4
:100050000C94AB030C94AB030C94AB030C94AB0368
:100060000C94AB030C94AB03506F636B6574204529
:100070006D70697265730080007B00517569740052
:10008000526573756D65000808FC848884A2D10AE6
:10009000044661696C656420746F206372656174E5
:1000A0006520756E697421004661696C6564207411
:1000B0006F20637265617465206275696C64696E36
:1000C00067210018181F80007E0000F80000F00073
:1000D00000E00000E00004E00004E00004E2E004CE
:1000E000E28004E28004E28004E28004E28004E230
:1000F000E004E0600CE00010E00000E00000E0013F
:1001000080F00180F801807E01801F818018180333
:10011000FFC00C003037FFEC780016AFFFF5A800E9
:1001200015A8FF15A88115A8FFD5AB8155AAA5D59F
:10013000AB8155AAA555AB81D5A89915A8FF15A6E1
:10014000006591C3898C423183C3C1404202304271
:100150000C0C423003C3C018180000000000FEFE63
:1001600000FEFE003E3E00FEFE00FEFE001E1E00E3
:100170001E1E001E1E001E1E001E1E001E1E001E35
:100180001E001E1E001E1E001E1E001E1E001E1E25
:1001900000FEFE00FEFE003E3E00FEFE00FEFE00F3
:1001A000FE1818E700E7BD00BDE7FFE7BD00BD8111
:1001B000FF81E700E7A500A5BDFFBDA500A5A5003F
:1001C000A5A500A5A500A5A500A5A500A5A500A518
:1001D000A500A5E700E7BD00BDE7FFE7BD00BD81C5
:1001E000FF81811881812481FFFFFF0808003C42C4
:1001F00099A5661800080860BCC299A5671D02256C
:100200000214020C02070251756974004F70746980
:100210006F6E73004D756C7469706C6179657220D6
:1002200067616D650053696E676C6520706C6179FC
:1002300065722067616D6500030307050705040506
:100240000504050306030207020201020203020E6F
:10025000090E0E0D0E0E0F0E070507050307050FFD
:10026000050705070607010205020007020207004D
:100270000207020002070200070603060707020240
:10028000050502010202040200050202050006073C
:1002900005050705020302020602000000000B002C
:1002A000030003070507040701050205070704000B
:1002B0000300000705050700050005020702000C02
:1002C00000020202000400040201070507050704FA
:1002D00001070405070203020704070107060601D8
:1002E0000107070707030307000500000D000205CB
:1002F000000505050005020107030F0903060306B3
:10030000070702020505070702070705070301079C
:10031000050607020705070504040307020507048D
:10032000040703070701060705070703030705037B
:100330000703060407010107010704070304030775
:100340000607050205010601010704000705010271
:10035000040507000201020808080003000603065E
:10036000070702020505070502070705070301073E
:10037000050607020705070504040307020507042D
:10038000040703070701060705070703030705031B
:100390000703060407010107010704070304030715
:1003A000060705020501060101070402070500070B
:1003B0000005070206020307050703053F213F1258
:1003C00008120A100A0E1C0E0C1E0C141A14161F0A
:1003D000161E131E1E1B1E1E1F1E3F213F3A2F3AC4
:1003E000173D173F213F181F02040A041F0E040483
:1003F0000E1F0A1F0A0E0E1F04110E2E252E2F2A65
:100400002E262929021F02081F08150E04040E15A6
:100410000E15151B151B040604040C040000000037
:1004200017000300031F0A1F16371A1904130A15B1
:100430003A000300000E11110E000A040A040E0413
:100440000030000404040010001804031F111F12E0
:100450001F101D151711151F07041F17151D1F1538
:100460001D01011F1F151F17151F000A0000320074
:10047000040A110A0A0A110A040115020E11171EB4
:10048000051E1F150A0E110A1F110E1F15111F053B
:10049000010E111D1F041F111F1108100F1F041B37
:1004A0001F10101F061F1E040F0E110E1F09060E2F
:1004B000112E1F051A121509011F011F101F0F18F9
:1004C0000F1F0C1F1B041B031C03191513001F1106
:1004D000030418111F000201022020200001020C59
:1004E000121E1F120C0C12120C121F0C1A14041ED6
:1004F00005242A1E1F021C141D1020201D1F081475
:10050000111F101E041E1E021C0C120C3E0A040CAD
:10051000123E1E040214160A020F120E101E0E10B6
:100520000E1E081E120C1226281E322A26041E2118
:10053000001F00211E040102013F213F0A4E6F20CF
:1005400053442063617264206F720A6E6F204C4FB7
:10055000414445522E4845580A0A153A457869746F
:10056000001D20466C617368696E670A20206C6FFD
:10057000616465722E2E2E0A0A444F4E2754205471
:1005800055524E204F464621000A0A153A49676ED9
:100590006F7265006D560A0A504C45415345205410
:1005A00055524E204F464620004C4F572042415452
:1005B0005445525921200017534400161378001651
:1005C0001314001510200015201000540A03E181B7
:1005D000867F3E186D830F0F0E0183866033186D82
:1005E000C3198F1803C38E6033186DE330CF18031F
:1005F000C39E603630CDE360CF3006C79E7E3E306E
:10060000CDB360CF300CC6F6603330D9B660CF338F
:10061000CFCCF66061B0DB1E60CF30D86CE6C06135
:10062000B0DB1E618F19986CC6C063B19B0E330F8F
:100630000FB078C6FF7E1F1B061E0F05008930080D
:10064000023802497868140000F6E8DBCFC3B8AE80
:10065000A49B928A827B746E68625C57524E4945B5
:10066000413E3A3734312E2C29272523211F1D1CCA
:100670001A1917161514131211100F0E0D0C0B0A60
:1006800009080706450068010000050068013801F7
:1006900000000500380168010000A2069E06010165
:1006A000FF030101F703000000070002010000033F
:1006B00004060000000000000000010204081020F1
:1006C00040800102040810200102040810200404E4
:1006D00004040404040402020202020203030303EA
:1006E0000303000000002300260029000000000092
:1006F000250028002B0000000000240027002A000D
:10070000BE030E04120411241FBECFEFD8E0DEBFDB
:10071000CDBF11E0A0E0B1E0E4EDF2E502C005904C
:100720000D92AE35B107D9F727E0AEE5B1E001C0D3
:100730001D92A837B207E1F713E0C2E8D3E004C086
:100740002197FE010E94CE24C038D107C9F70E942C
:10075000AD030C945D290C9400000E9403210E94BB
:1007600095048EE591E00E949A1C68E670E08EE5A3
:1007700091E00E941D1C0E94CC0FF7CF1092AF0198
:100780001092AE0183E591E09093AD018093AC01AE
:1007900008958EEE91E00E94710781E08093EE0152
:1007A00087E890E09093ED018093EC0182E08093E4
:1007B000EB011092E9011092EA0186E28093E501D3
:1007C00084E18093E6010E940B0586E090E00E94A0
:1007D0001F06882349F042E067E770E08EE591E06C
:1007E0000E945819811108958EEE91E00E94CB0B62
:1007F0000E94530681110E9416040E94130588234B
:10080000E1F30E941D058EEE91E00E94070B85EE3C
:1008100091E00E942D050E943204D7CF8EEE91E028
:100820000C9463068EEE91E00C9464068091F404BF
:10083000811117C081E08093F4043091F504209178
:10084000F6048091F7048091F8048091F904809176
:10085000FA048091FB048091FC04832F922F0C9466
:100860005E2608952091F5043091F6044091F70436
:100870005091F8046091F9047091FA048091FB049E
:100880009091FC04A1E00E94C2242093F5043093CF
:10089000F6044093F7045093F8046093F9047093BE
:1008A000FA048093FB049093FC0408958F929F9226
:1008B000AF92BF92CF92DF92EF92FF924B015C0119
:1008C00069017A010E945926BC01990F880B990B86
:1008D000C818D908EA08FB08A70196012F5F3F4F07
:1008E0004F4F5F4F0E947624680D791D8A1D9B1D16
:1008F000FF90EF90DF90CF90BF90AF909F908F9040
:100900000895E2E9F4E013861286118610861082BB
:1009100011821282138214821582168217823C96EB
:1009200084E0E23FF80779F708951092F5041092F9
:10093000F6041092F7041092F8041092F904109241
:10094000FA041092FB041092FC041092F3040E942B
:1009500081041092F2040895EF92FF920F931F9377
:10096000CF93DF93CDB7DEB72C970FB6F894DEBFE9
:100970000FBECDBF49835A836B837C839E83EF82F6
:10098000F88609871A873C8769817A814F81588563
:10099000240F352F311D62177307C8F4860F972F68
:1009A000911D4817590798F46B817C8149855A85B8
:1009B0008C85840F952F911D6817790740F42E813F
:1009C000260F372F311D81E04217530708F080E0D2
:1009D00081702C960FB6F894DEBF0FBECDBFDF91AD
:1009E000CF911F910F91FF90EF90089550E0480F25
:1009F000511D87FD5A9557FD0CC0843554F430E0E5
:100A0000260F311D67FD3A9537FD03C081E0603345
:100A10000CF080E008951092B2016AEB73E08CEA6A
:100A200091E00C94C3158EE591E00E94A01891E02E
:100A3000811101C090E0892F089560E08CEA91E077
:100A40000E94C5108CEA91E00C94B410FC01238143
:100A50004281618180810C94F604EF920F931F9381
:100A6000CF93DF93EC01009701F10E9426058823C4
:100A7000E1F01091CC0140E06E818CEA91E00E949F
:100A800016112F813885ED800C81498168818CEAAF
:100A900091E00E94DC14612F8CEA91E0DF91CF910C
:100AA0001F910F91EF900C941211DF91CF911F9134
:100AB0000F91EF900895FC01849108950196FC0137
:100AC000849108954CE3BC018EE591E00C94781775
:100AD0000F931F93CF93DF938C01C091CA01D091E4
:100AE000CB0122974093B5012093B6018CEA91E0A7
:100AF0000E94C31540E061E08CEA91E00E9416116B
:100B0000B8018CEA91E00E94CC22209749F0BE0106
:100B10008CEA91E0DF91CF911F910F910C94C31556
:100B2000DF91CF911F910F910895FF920F931F9323
:100B3000CF93DF93D82F162FC42FF22E242F0E948D
:100B4000F6048823C1F00091CC016F2D8CEA91E06E
:100B50000E9412112C2F412F6D2F8CEA91E00E94E0
:100B6000A311602F8CEA91E0DF91CF911F910F913B
:100B7000FF900C941211DF91CF911F910F91FF9074
:100B80000895EF92FF920F931F93CF93DF93C82F97
:100B9000D62F142FF22E0E94F6048823D1F0E09075
:100BA000CC01602F8CEA91E00E9412110F2D212FB1
:100BB0004D2F6C2F8CEA91E00E9452116E2D8CEA21
:100BC00091E0DF91CF911F910F91FF90EF900C94E6
:100BD0001211DF91CF911F910F91FF90EF90089527
:100BE000EF92FF920F931F93CF93DF93C82FD62FCF
:100BF000142FF22E0E94F6048823D1F0E090CC014D
:100C0000602F8CEA91E00E9412110F2D212F4D2FA1
:100C10006C2F8CEA91E00E947A116E2D8CEA91E0A3
:100C2000DF91CF911F910F91FF90EF900C941211D3
:100C3000DF91CF911F910F91FF90EF900895682F52
:100C400088E691E00E94221091E0811101C090E0BD
:100C5000892F0895CF93C62F682F88E691E00E94D0
:100C6000411091E0C81708F090E0892FCF910895C6
:100C700060E00C942A0681E090E00E943806811121
:100C800010C083E090E00E94380681110AC090E015
:100C900080E00E943806811104C082E090E00C944C
:100CA000380681E008950E943B0681110AC084E065
:100CB00090E00E943806811104C085E090E00C9419
:100CC000380681E00895089508950F931F93CF93F8
:100CD000DF93CDB7DEB728970FB6F894DEBF0FBE0F
:100CE000CDBF162F00E028E044E56BE280E00E94D3
:100CF000F0051F921F9386E091E09F938F931F92C0
:100D000088E08F938E010F5F1F4F1F930F930E94F8
:100D100070262CE244E068E372E0C8010E94680596
:100D20000FB6F894DEBF0FBECDBF28960FB6F8946D
:100D3000DEBF0FBECDBFDF91CF911F910F91089500
:100D4000CF92DF92FF920F931F93CF93DF93CDB794
:100D5000DEB760970FB6F894DEBF0FBECDBF6C0153
:100D600060E08CEA91E00E94121105E024E540E089
:100D700060E08CEA91E00E947A11F60181891F926D
:100D80008F938CE091E09F938F931F9280E1F82ED8
:100D9000FF928E010F5F1F4F1F930F930E947026CB
:100DA00021E042E068E372E0C8010E946805F601B4
:100DB00082891F928F9381E191E09F938F931F927D
:100DC000FF921F930F930E94702621E046E168E393
:100DD00072E0C8010E946805F60183891F928F9313
:100DE00086E191E09F938F931F92FF921F930F9341
:100DF0000E94702621E04AE268E372E0C8010E9486
:100E000068050FB6F894DEBF0FBECDBF60960FB673
:100E1000F894DEBF0FBECDBFDF91CF911F910F9130
:100E2000FF90DF90CF900895CF92DF92EF92FF92E4
:100E30000F931F93CF93DF9300D000D000D0CDB796
:100E4000DEB76B0109831A832B833C837C012CE67C
:100E5000E21A2DEFF20AF7014081403208F03FC05C
:100E600054E1242F30E08C01549F000D111D1124FA
:100E7000F801658F2F5F3F4F529FB001539F700D58
:100E80001124860F971F29813A81FC013183208329
:100E90008B819C81F801978B868B8C2D0E947C0E18
:100EA000F801848F81E083A3F2E0CF16D1040CF423
:100EB00080E0F80181A3F70180818F5F808381E06A
:100EC00026960FB6F894DEBF0FBECDBFDF91CF914F
:100ED0001F910F91FF90EF90DF90CF90089580E0E9
:100EE000EFCFEF92FF920F931F93CF93DF9300D03A
:100EF00000D000D0CDB7DEB77C018C010C561D4F61
:100F0000D8011C92FC01E256FD4F8FEF8083C70190
:100F10008B569D4F0E94ED0B0E94D60CF7017496E4
:100F200084E1DF01982F1D929A95E9F77496E017F6
:100F3000F107B9F789E1D70151968C93519782E374
:100F400052968C9352978BE453968C9324E130E025
:100F500040E050E060E070E0CB010E9456047A83EC
:100F6000698324E130E040E050E060E070E0CB01D4
:100F70000E945604262F7C836B8309811A813C8151
:100F80004D815E8164E070E0C7010E941407811109
:100F900004C088EA90E00E94620528E330E040E067
:100FA00050E060E370E080E090E00E9456047A83B5
:100FB000698328E330E040E050E060E370E080E0E7
:100FC00090E00E9456047C836B8380E00E944A0D6F
:100FD0008D8380E00E94540DF701EF55FD4F108284
:100FE00031961082329710823397108209811A81CC
:100FF0002B813C814D81582F70E060E0C7010E9439
:101000001407811110C081E990E026960FB6F8947C
:10101000DEBF0FBECDBFDF91CF911F910F91FF902B
:10102000EF900C94620526960FB6F894DEBF0FBEC3
:10103000CDBFDF91CF911F910F91FF90EF90089559
:10104000CF93DF9300D000D000D0CDB7DEB7FC0146
:10105000E956FD4F2081318144E150E0421B530BA2
:101060008B569D4FFC018081918126E230E0281B48
:10107000390B3A8329835C834B833A815C8168E036
:1010800078E080E090E026960FB6F894DEBF0FBEC1
:10109000CDBFDF91CF9108953F924F925F926F92B3
:1010A0007F928F929F92AF92BF92CF92DF92EF92F8
:1010B000FF920F931F93CF93DF9300D000D000D007
:1010C000CDB7DEB75C018C01912C88248A9444242E
:1010D0004A94542C3201F80183A1882309F444C0B6
:1010E00084A1811141C0C5010E94200829833A834F
:1010F0004B835C836D837E83F801C488D588E68842
:10110000F788858D0E944A0D382EF801858D0E9442
:10111000540D29813A81C21AD30A232D30E0359526
:101120002795C20ED31E2B813C81E21AF30A90E070
:1011300095958795E80EF91ECC9CC001CD9C900D2D
:10114000900D1124EE9C9001EF9C300D300D112478
:10115000820F931FB0E0A0E084159505A605B705A2
:1011600018F4892C2C013D010C5E1F4F9394F0E282
:101170009F12B1CFF501E256FD4F808226960FB641
:10118000F894DEBF0FBECDBFDF91CF911F910F91BD
:10119000FF90EF90DF90CF90BF90AF909F908F9097
:1011A0007F906F905F904F903F900895FC01E356C1
:1011B000FD4F2081222351F033962081211106C05A
:1011C00031968081853010F48F5F808308958F92EF
:1011D0009F92BF92CF92DF92EF92FF920F931F9355
:1011E000CF93DF9300D000D000D0CDB7DEB77C0125
:1011F0004B016A01FB0181850E944A0D182FF40101
:1012000081850E94540DB82EF4010081812F90E059
:101210009C0135952795280F391F032E000C440B90
:10122000550B612F70E090E080E00E945604060F9D
:10123000F40112818B2D90E09C0135952795280FA4
:10124000391F032E000C440B550B6B2D70E090E002
:1012500080E00E9456041E821D82802F90E09A83B7
:101260008983160F612F70E0212F7C836B831A8195
:101270003C8140E05E81B601C7010E9414072696BA
:101280000FB6F894DEBF0FBECDBFDF91CF911F9197
:101290000F91FF90EF90DF90CF90BF909F908F9035
:1012A0000895CF92DF92EF92FF920F931F93CF9307
:1012B000DF9300D000D000D0CDB7DEB77C016A014B
:1012C0000E94200889019A01AB01B601C7010E9462
:1012D000140726960FB6F894DEBF0FBECDBFDF9180
:1012E000CF911F910F91FF90EF90DF90CF900895D5
:1012F0000F931F93CF93DF93EC01CF55DD4F2881E0
:101300008C0100561D4F253018F5FC01E256FD4FAB
:1013100020812F3F81F0FC0134E12302E00DF11D1B
:10132000112421E024A3FC01E356FD4F20838E55B8
:101330009D4FFC011082188281E09881953008F45D
:1013400080E0F8018083DF91CF911F910F91089584
:10135000F8012081222381F3FC0130E020E044A148
:101360002F5F3F4F4423E1F044E1429FB001439F90
:10137000700D1124680F791FFC01ED55FD4F10828F
:1013800031972081222339F02230B1F650E040E03D
:101390000E94E708D1CF42E050E00E945109CCCF33
:1013A000749620323105D9F6C7CFCF93DF93EC0185
:1013B000C356DD4F28812223D9F0DC01A156BD4F51
:1013C0002C912530C0F0FC019C0120583D4F44A1D8
:1013D000411114A27496E217F307C9F71C92188200
:1013E000FC01E056FD4F10828F559D4FFC0110828D
:1013F000DF91CF9108952F5F2C93FACFCF92DF9298
:10140000EF92FF920F931F93CF93DF9300D000D002
:1014100000D0CDB7DEB78C01FC01E356FD4F8081D3
:10142000882309F1C8010E94200829833A834B834D
:101430005C836D837E83F801680120E8C21A2DEF7A
:10144000D20A84A19F012C5E3F4F7901882339F095
:101450004B815C8169817A81C9010E94820EF7010A
:10146000EC14FD0471F7F801E156FD4F1082269649
:101470000FB6F894DEBF0FBECDBFDF91CF911F91A5
:101480000F91FF90EF90DF90CF900895EF92FF9231
:101490000F931F93CF93DF93FC01E056FD4F208104
:1014A000222349F1EC017C0180E8E81A8DEFF80A6B
:1014B0008E010E551D4F8CA164968823C9F0CE0174
:1014C0000E94B00FF80140819FEF940F282F30E069
:1014D000491771F0993008F097E0B901092E02C060
:1014E000759567950A94E2F760FF0CC0F801908348
:1014F000CE15DF0501F7DF91CF911F910F91FF907E
:10150000EF9008959150E4CFEF92FF920F931F93C5
:10151000CF93DF93FC01E056FD4F2081222349F158
:10152000EC017C0180E8E81A8DEFF80A8E010E5577
:101530001D4F8CA164968823C9F0CE010E94B00F84
:10154000F801408191E0940F282F30E0491771F0A5
:10155000983008F090E0B901092E02C075956795A2
:101560000A94E2F760FF0CC0F8019083CE15DF0506
:1015700001F7DF91CF911F910F91FF90EF900895A8
:101580009F5FE4CF0F931F93CF93DF93EC01FC0198
:10159000E056FD4F80818823A9F1FE0190E080E0B4
:1015A00024A10196222351F144E1489F9001499FD3
:1015B000300D1124CE01820F931F0E94B00F90E0D6
:1015C0008E010E551D4FF801208102C0959587951B
:1015D0002A95E2F780FD03C0CE010E94840AF8013B
:1015E000808190E00E94B80F2CE248E268E372E04C
:1015F000DF91CF911F910F910C9468057496803202
:10160000910571F6DF91CF911F910F9108958F92FF
:101610009F92AF92BF92CF92DF92EF92FF920F9381
:101620001F93CF93DF93EC018C010C5E1F4FF12CC5
:10163000E12C912C6C0182E6C81A8DEFD80A5E016C
:10164000EBE6AE1AEDEFBE0AF80187858823D9F0E4
:10165000F60180818F3F39F0082E000C990B41E094
:101660008E159F0509F040E0B501C8010E945E0D8E
:10167000F8018088882039F0911005C06085CE017E
:101680000E946506982CFFEFEF1AFF0A0C5E1F4FB1
:1016900080E2E816F104C1F68881882339F19920A7
:1016A00099F001E023E04AE06CE284E40E94C10585
:1016B000FE01EF55FD4F4081442331F0440F23E0FC
:1016C0006CE284E40E94F005CE010E94C20ACE01C1
:1016D000DF91CF911F910F91FF90EF90DF90CF900E
:1016E000BF90AF909F908F900C94A006DF91CF9108
:1016F0001F910F91FF90EF90DF90CF90BF90AF9030
:101700009F908F900895CF93DF93EC0184E090E059
:101710000E943806882329F0CE01DF91CF910C94E6
:10172000D60884E090E00E941F06882329F0CE01AD
:10173000DF91CF910C94780985E090E00E94380603
:10174000882329F0CE01DF91CF910C94D50985E053
:1017500090E00E941F06882329F0CE01DF91CF91EF
:101760000C94FE0990E080E00E941F06882329F077
:10177000CE01DF91CF910C94460A82E090E00E9466
:101780001F06882329F0CE01DF91CF910C94840AA3
:10179000DF91CF9108950F931F93CF93DF93EC01C7
:1017A0008C010B561D4FFC01E056FD4F6081C801B6
:1017B0000E94D30CC8010E94350CCE010E944C0837
:1017C00060E270E0CE0144960E948A0ECE01DF9165
:1017D000CF911F910F910C94830BFC011182108209
:1017E000138212821482158283E086831782089501
:1017F000CF93DF93CDB7DEB72C970FB6F894DEBF4B
:101800000FBECDBF1C861B86FC0122813381420F97
:10181000531F80819181680F791F78876F835A8762
:10182000498786E0FE013796DE01119601900D9200
:101830008A95E1F729813A814B815C816D817E81B6
:1018400080E090E02C960FB6F894DEBF0FBECDBFBF
:10185000DF91CF910895FC019081490FDB014C93FA
:101860008281280F11962C930895CF93DF93EC017A
:101870008F81882319F01C821D821BC08E818330CA
:10188000D8F48F5F8E832C8188819981820F911D7E
:1018900027FD9A9597FF80C0998388832D818A813F
:1018A0009B81820F911D27FD9A9597FF79C09B839D
:1018B0008A83DF91CF9108951E820E943B06882380
:1018C00069F190E080E00E943806882329F08C813D
:1018D00087FF47C08E5F8C8381E090E00E943806CE
:1018E000882329F08D8187FF41C08E5F8D8383E03F
:1018F00090E00E943806882331F08D8118160CF094
:101900003AC082508D8382E090E00E94380688239E
:1019100029F08C8118169CF582508C8390E080E031
:101920000E94380681110BC082E090E00E943806C8
:10193000811105C08C81181634F581508C8381E0AB
:1019400090E00E94380681119ECF83E090E00E94D3
:101950003806811198CF8D811816CCF481508D8373
:1019600092CF85300CF0B8CF8F5FB5CF85300CF0BB
:10197000BECF8F5FBBCF8C3F34F28150C3CF8C3F43
:101980006CF28150CACF8823D1F28F5FD7CF8823E2
:1019900009F479CF8F5FE3CF198218821C827ECF42
:1019A0001B821A8269CFFC0167830895FF920F930F
:1019B0001F93CF93DF9303E315E08BEE91E0F801E3
:1019C000908787830E945B05F80182838BEE91E00C
:1019D0000E945E05F801838315821482FF24F3942C
:1019E000F682CDEFD4E085EF91E098878F830E9457
:1019F0005B058A8385EF91E00E945E058B831D82E3
:101A00001C82FE8281EA91E0F801928F818F0E9410
:101A10005B05F801848B81EA91E00E945E05F80184
:101A2000858B178A168AF08E8DE091E094A783A7A4
:101A30000E945B05F80186A38DE091E00E945E059F
:101A4000F80187A311A610A6F2A687E591E09A8F68
:101A5000898F0E945B058C8B87E591E00E945E0573
:101A60008D8B1F8A1E8A13E0188F83EC90E09CA751
:101A70008BA70E945B058EA383EC90E00E945E051D
:101A80008FA319A618A61AA7DF91CF911F910F91C6
:101A9000FF90089599E0899FF0011124ED5CFA4FC1
:101AA000878190850C945B0599E0899FF001112452
:101AB000ED5CFA4F878190850C945E058F929F9222
:101AC000AF92BF92CF92DF92EF92FF920F931F934C
:101AD000CF93DF9300D000D000D0CDB7DEB77C012C
:101AE0006B01842EDC011F968C911F97882309F4CB
:101AF00080C019969C90E92DF0E0B9E09B9E800192
:101B00001124D7011D968C911D978111B3C01E968B
:101B10008C91882309F480C003501B4FF801148274
:101B20001582882351F0D70153968C9153978F5F7C
:101B3000853008F074C053968C93D7011A968D9116
:101B40009C911B978130910509F48AC008F484C0E8
:101B50008230910509F46AC0039709F473C0F70154
:101B60002281338140815181B801C6010E942B0C32
:101B7000C8010E942D05811005C0D70150968C9197
:101B80008823B9F1F7014281538160817181C601D7
:101B90000E94F80B29833A834B835C83C980DA80E7
:101BA000AB80BC80D70150968C9101E0811101C0BF
:101BB00003E0892D0E944A0D182F892D0E94540D93
:101BC000F7019585992309F477C0282F2695269546
:101BD000280F412F46954695410F86958695869507
:101BE0006A2D681B1695169516958C2D811B0E94E3
:101BF000C10526960FB6F894DEBF0FBECDBFDF91AC
:101C0000CF911F910F91FF90EF90DF90CF90BF90F9
:101C1000AF909F908F9008950D5C1A4F7FCFF70182
:101C2000138A848591E08927848787CF82E0F80131
:101C30008583D7011C968C91882309F490CF83E08B
:101C400085838DCFF7018485882309F488CF81E0CF
:101C5000D80115968C9383CF81E0F8018483E8CF77
:101C600081E0F80184831C968C91882309F477CF56
:101C700082E0E6CFC80183509B4F5C01EE0FFF1F4F
:101C8000E95EFE4F818112962D913C911397280FAA
:101C9000311D87FD3A9580814D915C91480F511D12
:101CA00087FD5A95B501C6010E942B0CC5010E9403
:101CB0002D050D5C1A4F53CF682F66956A0D7B2D4D
:101CC000711D812F8695202F412F8C0D9D2D911DEB
:101CD00026960FB6F894DEBF0FBECDBFDF91CF9131
:101CE0001F910F91FF90EF90DF90CF90BF90AF903A
:101CF0009F908F900C949505E82FF0E0E75BFE4FE6
:101D000080810895FC01758364835783468381E055
:101D1000868708952F923F924F925F926F927F92A3
:101D20008F929F92AF92BF92CF92DF92EF92FF92EB
:101D30000F931F93CF93DF93CDB7DEB762970FB6A4
:101D4000F894DEBF0FBECDBF882E592E7E876D87DB
:101D5000C82ED92E312C212C8D859E85281639062A
:101D6000C9F462960FB6F894DEBF0FBECDBFDF9107
:101D7000CF911F910F91FF90EF90DF90CF90BF9088
:101D8000AF909F908F907F906F905F904F903F901B
:101D90002F900895D6011F968C911F97882309F4E0
:101DA000D8C01E96BC901E97BB2009F4D2C0ED91FE
:101DB000FC91119719968C91A82FB0E0AD5BBE4FA6
:101DC0004C90842D90E0D60114966D917C911597DE
:101DD0009F01281B390B6217730788F51B961C920D
:101DE0001E921A97942C9194D60112964D915C9163
:101DF000139716962D913C91DA01A81BB90B2A175F
:101E00003B0760F522E030E0F601338722874194FA
:101E1000D6011E96BC92BB2009F49BC0A82CB52C01
:101E2000712C612C292D092C000C330B388B2F873A
:101E3000842D042C000C990B9A8B898B28C09F0150
:101E4000280F391F912C2617370770F621E030E054
:101E50001B963C932E931A97942CC6CF840F951FF4
:101E60008217930740F4E3E0F0E0D6011B96FC9361
:101E7000EE931A97CDCF9E2E961A442E421AB12C6D
:101E8000C7CFBFEF6B1A7B0AE4E1AE0EB11CAD8584
:101E9000BE856A167B0609F448C0F60180819181EF
:101EA0002F853889820F931F98878F838281938132
:101EB000A989BA898A0F9B1F9A87898781850E9481
:101EC0004A0D8B87F60181850E94540D8C87D501C0
:101ED0001F968C911F978823A1F22614370489F24C
:101EE0008D919C9111979A8389839C838B831996FA
:101EF0008C910E944A0D8D83F50181850E94540DBD
:101F00008E83E980FA800B811C812D81382F4F81CF
:101F1000588569857A858B859C850E94AC048823C9
:101F200009F4AFCFD6011E961C92F6018685882350
:101F300081F080819181890D911D97FC9A95918303
:101F4000808382819381840D911D47FC9A959383B0
:101F50008283FFEF2F1A3F0A24E1C20ED11CFCCE70
:101F6000DC011996EC91F0E0EF5DFE4F8081089561
:101F7000880F991FFC01E35CFE4F808191810895D9
:101F8000BC016F5F7F4F80E1FB0111928A95E9F7F9
:101F90008EE591E00C94F51C43E06FEF71E08EE567
:101FA00091E00E945819811106C08EEE91E00E94C6
:101FB000C00F0C94C9030895FC0188E0808389E078
:101FC000818387E0828386E0838384E0848382E068
:101FD000858381E186830895FF920F931F93CF93AA
:101FE000DF93EC018C01095F1F4FFF24FA9462E03C
:101FF00088810E94DF2188810E9449222F81892BBC
:1020000081F42F5F2F8360E088810E94DF21219679
:10201000C017D10761F7DF91CF911F910F91FF900A
:1020200008952223A1F32F3F11F41F82ECCFFF82EA
:10203000EACFFC01E60FF11D81E09781913009F0B4
:1020400080E00895FC01E60FF11D81E097819F3F3C
:1020500009F080E00895860F911DFC0187814230D0
:1020600038F49FEF980F81E09E3F50F080E008C069
:102070008F3FE1F3642F0E94422481E09130B1F759
:102080000895860F911DFC0187818F3F09F480E040
:1020900008958EBD0DB407FEFDCF8EB50895DC0109
:1020A000643508F042C0403308F03FC090968C91F0
:1020B0009097E62F062E000CFF0B242F25952595D3
:1020C000259594E52902E00DF11D1124E759FA4FF9
:1020D0002081342F37708230A1F4822F90E0032EBC
:1020E00002C0959587950A94E2F7809581708823C0
:1020F00099F081E090E001C0880F3A95EAF7822BD1
:1021000013C08330A1F71C968C916427062E000C17
:10211000770B682760FDEDCF81E090E001C0880F6C
:102120003A95EAF780958223808308951F93CF9391
:10213000DF93EC01162FF89460E08F850E941B223C
:10214000888918161CF460E00E941B22812F0E94CF
:102150004910888918161CF461E00E941B227894AB
:10216000DF91CF911F910895E9E6F5E028EF31E086
:10217000DF01A9011D9241505040E1F7DC011996A1
:102180001C9219971A961C92089548EF51E06FEF30
:102190007FEF89E695E00C946926CF92DF92EF926B
:1021A000FF920F931F93CF93DF93EC018C858F5F8A
:1021B0008C8789E6E82E85E0F82E10E0612F6064B8
:1021C000CE010E94961060E8CE010E94961061E058
:1021D0008F850E941B22888918161CF460E00E94DB
:1021E0001B22670104E5F60181916F010E944910ED
:1021F0000150C9F7888918161CF461E00E941B225F
:102200001F5FF4E5EF0EF11C1630C1F660E4CE015D
:10221000DF91CF911F910F91FF90EF90DF90CF90C2
:102220000C949610FC0160A361A30895FC0160A3C7
:1022300041A30895EF92FF920F931F93CF93DF93E3
:102240008C01D62FF42EE22EC0E0CE1544F44F2D93
:102250004C0F6D2FC8010E944F10CF5FF6CFDF915A
:10226000CF911F910F91FF90EF900895EF92FF9201
:102270000F931F93CF93DF938C01F62ED42FE22E72
:10228000C0E0CE1544F46F2D6C0F4D2FC8010E9495
:102290004F10CF5FF6CFDF91CF911F910F91FF903D
:1022A000EF900895EF92FF920F931F93CF93DF93D8
:1022B0007C01162FD42FC22F0E9436114FEF400FF2
:1022C0004D0F2C2F612FC7010E943611202F4D2F4B
:1022D000612FC7010E941A116FEF6C0F610F202F41
:1022E0004D2FC701DF91CF911F910F91FF90EF907C
:1022F0000C941A11DF92EF92FF920F931F93CF93DA
:10230000DF937C01D62FD22EC42F002E000C110B90
:10231000040F111D47FD1A958C2F0C2E000C990BE4
:102320008017910744F42D2D4C2F6D2FC7010E946B
:102330003611CF5FF1CFDF91CF911F910F91FF90B9
:10234000EF90DF9008959F92AF92BF92CF92DF926D
:10235000EF92FF920F931F93CF93DF938C01E62EA2
:10236000F42EC22F81E0D82ED21AC22EC194CC0CEA
:10237000422F4F0DC8010E944F104F2D4C1B6E2D48
:10238000C8010E944F106C2F6E0D4F2DC8010E9486
:102390004F106E2D6C1B4F2DC8010E944F10D0E0C6
:1023A000DC170CF044C0D7FC04C0C150C394C394E4
:1023B000DC0CDF5F8D2F880F8F5FD80E9E2C9D0E5B
:1023C000BF2CBC0E4B2D692DC8010E944F10AE2CA6
:1023D000AD1A4B2D6A2DC8010E944F10BF2CBC1A9C
:1023E0004B2D692DC8010E944F104B2D6A2DC8013D
:1023F0000E944F10BF2CBD0E4B2DAE2CAC0E6A2D83
:10240000C8010E944F104B2DBE2CBC1A6B2DC80169
:102410000E944F109F2C9D1A492D6A2DC8010E94C1
:102420004F10492D6B2DC8010E944F10B9CFDF917D
:10243000CF911F910F91FF90EF90DF90CF90BF90C1
:10244000AF909F9008958F929F92AF92BF92CF923C
:10245000DF92EF92FF920F931F93CF93DF937C0154
:10246000162FD42EC22F81E0C82EC21AB22EB194DC
:10247000BB0CD0E0802F8470A82E802F8270982E05
:10248000802F8870882E0170DC170CF04DC0C7FCBF
:1024900004C0C150B394B394CB0CDF5F8D2F880F71
:1024A0008F5FC80EAA2071F04D2D4C0F612F6D0F5C
:1024B000C7010E944F104D2D4D0F6C2F610FC701AA
:1024C0000E944F10992071F04D2D4C1B612F6D0F04
:1024D000C7010E944F104D2D4D1B6C2F610FC7017E
:1024E0000E944F10882071F04D2D4D0F612F6C1BF5
:1024F000C7010E944F104D2D4C0F612F6D1BC7015E
:102500000E944F10002309F4BFCF4D2D4D1B612FAA
:102510006C1BC7010E944F104D2D4C1B612F6D1B72
:10252000C7010E944F10B0CFDF91CF911F910F9143
:10253000FF90EF90DF90CF90BF90AF909F908F90E3
:1025400008957F928F929F92AF92BF92CF92DF9227
:10255000EF92FF920F931F93CF93DF935C01C62EF0
:10256000942EC22F11E0121BD22ED194DD0C83E0E9
:10257000F82ED0E0802F8170782E882483948E0CE2
:102580000270DC17ACF517FD04C0C150D394D3948E
:102590001D0DDF5F1F0D772099F02C2F220F280DC6
:1025A000492D4C1B6C2D6D0FC5010E941A112E2D4B
:1025B0002F0D492D4D1B6C2F6C0DC5010E941A115A
:1025C000002399F02C2F220F280D492D4C1B6C2D28
:1025D0006D1BC5010E941A112E2D2F0D492D4D1B6B
:1025E0006C2D6C1BC5010E941A11F394F394C9CF92
:1025F000DF91CF911F910F91FF90EF90DF90CF90DF
:10260000BF90AF909F908F907F9008959F92AF92D0
:10261000BF92CF92DF92EF92FF920F931F93CF93CF
:10262000DF93EC01B62E142FD22EAE2CAA0C922ED4
:102630009A18CE2CC60E292D6C2D0E943611FF241F
:10264000FA94F00EF10E292D4F2D6C2DCE010E9423
:1026500036110A191E0D202F412F6B2DCE010E941D
:102660001A11DB0C6FEF6D0D202F412FCE010E9450
:102670001A1101E02E2D412F6C2DCE010E94231244
:102680008E2D8095D80E02E02E2D412F6D2DCE017E
:102690000E942312FE1804E02E2D4F2D6D2DCE0129
:1026A0000E94231208E02E2D4F2D6C2DCE010E948A
:1026B0002312DF91CF911F910F91FF90EF90DF9048
:1026C000CF90BF90AF909F900895AF92BF92CF925E
:1026D000DF92EF92FF920F931F93CF93DF936C01E2
:1026E000C62FF42EA22ED02F1E2DEE0CB12EB60E1C
:1026F0002E196B2D0E947A11D150DE19F10E6FEF59
:102700006C0F6A0D611BED2E01E0212F4F2DC601CC
:102710000E94A11202E0212F4F2D6B2DC6010E94B5
:10272000A112DF91CF911F910F91FF90EF90DF9059
:10273000CF90BF90AF9008952F923F925F926F928B
:102740007F928F929F92AF92BF92CF92DF92EF9241
:10275000FF920F931F93CF93DF93EC01F901E49065
:102760003196849164350CF015C10E2C000CFF08D5
:10277000062F062E000C110BF701E00FF11F1E169D
:102780001F060CF007C140330CF004C1A82FC42E63
:10279000042E000CDD085601A80EB11C87FDBA946A
:1027A0001A141B040CF0F6C02E5F3F4F570197E040
:1027B000A90EB11CB7FE04C05701BEE0AB0EB11CA0
:1027C000B3E0B594A794BA95E1F747FF0AC0A42FE8
:1027D000A80FAC9CC001AD9C900D1124281B390B97
:1027E00040E08A2F0A2E000C990B840F911D47FDA3
:1027F0009A95C19714F0A0E3A41BF8A067FD60E0D0
:10280000E535F10514F0E4E5F0E09E2FCC85C42712
:10281000C62E062E000CDD08F601E01BF10B8F0121
:102820004F01F7E08F229924E0E8F0E002C0F5952F
:10283000E7958A94E2F77E2F17FF02C0095F1F4FCA
:10284000F3E015950795FA95E1F7200F311F542F06
:10285000577081E001C0880F5A95EAF74595459574
:102860004595F601B4E54B02E00DF11D1124AF01D1
:1028700047595A4FD0E02A2EAA0F3308EE24E3948A
:10288000BB24D21513040CF085C0F9015490F1E07B
:10289000FF121AC06901962E8A01E72F991608F0D7
:1028A00057C08E2E852021F0D8018C90882A8C92DA
:1028B000E69531F4BFEFCB1ADB0AF6015490E0E85D
:1028C00093940F5F1F4FEACFF1101CC0782E7094C5
:1028D0006901962E8A01E72F991608F039C08E2ECD
:1028E000852021F0D8018C9087208C92E69531F4D8
:1028F000BFEFCB1ADB0AF6015490E0E893940F5F28
:102900001F4FEACFF3E0FF122CC0782E70946901BC
:10291000862E8A01972E8916D0F4E92DE52141F003
:10292000D801EC916C2E682460FE0FC0E82BEC936C
:10293000969439F4BFEFCB1ADB0AF6015490E0E825
:102940009E2E83940F5F1F4FE6CFE721F0CFCE2559
:10295000880F19F44C5A5F4F81E0DF5F2A0D3B1D51
:1029600090CF6901962E8A01E72F991688F78E2E4F
:10297000852021F0D8018C9088268C92E69531F440
:10298000BFEFCB1ADB0AF6015490E0E893940F5F97
:102990001F4FEBCFDF91CF911F910F91FF90EF90E1
:1029A000DF90CF90BF90AF909F908F907F906F906F
:1029B0005F903F902F9008952F923F924F925F9299
:1029C0006F927F928F929F92AF92BF92CF92DF923F
:1029D000EF92FF920F931F93CF93DF9300D000D01D
:1029E00000D01F92CDB7DEB74C01462E342E6901C0
:1029F0008E2D01111DC0E1101BC0C40127960FB61A
:102A0000F894DEBF0FBECDBFDF91CF911F910F9124
:102A1000FF90EF90DF90CF90BF90AF909F908F90FE
:102A20007F906F905F904F903F902F900C949C13ED
:102A3000F60154903196E490A52CB12C9501295FB4
:102A40003F4FA90133E0559547953A95E1F75B83F0
:102A50004A830370F12CEE2DF0E0FD83EC835A9451
:102A60001FEF1E0D2F2D0F2C000C330B2A153B05CD
:102A70000CF070C0F982F7FE03C0F7E0FF0DF98398
:102A8000298125952595259529839F2D977897FF51
:102A900003C09150986F9F5F20E8622E712C02C096
:102AA000759467949A95E2F7212C4981042E000CC5
:102AB000550B4E5F5F4F5F834E83222D022C000C1F
:102AC000330BEC81FD812E173F070CF041C04A818A
:102AD0005B81429FF001439FF00D529FF00D112446
:102AE0002E813F81E20FF31FEC0DFD1DE491F0E01C
:102AF000E621F721EF2B41F1023069F0612F6219D5
:102B00004F2D033061F0452D4F19622D013039F002
:102B1000422D6F2D04C0652D6F19412F4219882356
:102B2000A9F0382F3370398380FF03C0552D561B11
:102B3000652F81FF03C08E2D841B482F640D430D2C
:102B4000C4010E944F1089812394B7CF1982F6CF18
:102B5000F39488CF27960FB6F894DEBF0FBECDBF93
:102B6000DF91CF911F910F91FF90EF90DF90CF9069
:102B7000BF90AF909F908F907F906F905F904F909D
:102B80003F902F900895DC01FB0184918F5F149694
:102B90008C9314973196E491EF5F1596EC9315970B
:102BA0006E5F7F4F5F967C936E935E970895EF9272
:102BB0000F93CF93DF93EC014E876D872F87E98AC0
:102BC000088B81E0888788A319A28F836AEB73E062
:102BD000CE010E94C3150E94FF2381E00E941524AC
:102BE00085E00E9423248CE00E941E2461E08E85F3
:102BF0000E94DF2161E08D850E94DF2161E08F85E9
:102C00000E94DF21898918161CF461E00E94DF21EF
:102C1000888918161CF461E00E94DF218989181642
:102C20006CF460E00E941B226AE070E080E090E0BB
:102C30000E94DD2061E089890E941B228D85082E7B
:102C4000000C990BFC01E253F94FE491F0E0EE0F18
:102C5000FF1FE451F94F259134913D8B2C8BFC01E2
:102C6000E654F94FE491EB8F8E85082E000C990BFA
:102C7000FC01E253F94FE491F0E0EE0FFF1FE45145
:102C8000F94F259134913B8B2A8BFC01E654F94F87
:102C9000E491EA8F8889082E000C990BFC01E2531D
:102CA000F94FE491F0E0EE0FFF1FE451F94F259149
:102CB00034913F8B2E8BFC01E654F94FE491EC8F5D
:102CC0008F85082E000C990BFC01E253F94FE4911B
:102CD000F0E0EE0FFF1FE451F94F25913491398F49
:102CE000288FFC01E654F94FE491ED8F61E2CE01AB
:102CF0000E94961064E1CE010E9496108B8587FF9A
:102D000002C08FE78B876B856068CE010E949610AA
:102D100060E2CE010E9496106CE0CE010E949610F7
:102D2000CE01DF91CF910F91EF900C94CD104F9287
:102D30005F926F927F928F929F92AF92BF92CF924B
:102D4000DF92EF92FF920F931F93CF93DF93EC01EB
:102D5000862EF42E102F83E586170CF485C08FE2A3
:102D600084170CF481C04C814150550B049FC00165
:102D7000059F900D1124860F911D67FD9A951816D9
:102D800019060CF071C03D818F2D0F2C000C990B92
:102D9000039F800D911D1124181619060CF064C0B4
:102DA00078A0E62E912CC22ED12C292D092C000CB6
:102DB000330B8C8190E0281739070CF054C0019731
:102DC000E0E02817390771F0C89EF001C99EF00DA8
:102DD000D89EF00D11242E0F3F1FEE8DFF8DE20FB8
:102DE000F31FE4915F2C612C492C480C2D81862D1A
:102DF000062C000C990B2817190691F18CF1AE2EB8
:102E0000B12CE0FF16C0113061F4462D4F0D642D3A
:102E1000CE010E944F10F501F595E7956394510E90
:102E2000E5CF012F212F452D6E2DCE010E947A1165
:102E3000F2CF89A198A1891771F388A3113041F4C9
:102E4000462D4F0D642DCE010E944F1078A2E3CF86
:102E5000012F212F452D6E2DCE010E947A11F6CF24
:102E60009394E10EA2CF78A2DF91CF911F910F91A1
:102E7000FF90EF90DF90CF90BF90AF909F908F909A
:102E80007F906F905F904F9008950F93CF93DF9353
:102E9000EC01262F6A3049F428859D818A85299F77
:102EA000800D11248A8719861DC06D30D9F00885E0
:102EB0004A8569850E94971628853C818985239FCC
:102EC000800D112489879F81992361F0082E000CC1
:102ED000990B44E550E0239F4019510911244817EC
:102EE0005907DCF281E090E0DF91CF910F910895D6
:102EF000FC01EC57FF4F718360838A579F4F445FFB
:102F0000FC01408308956F927F928F929F92AF92BF
:102F1000BF92CF92DF92EF920F93CF93DF934C014A
:102F20005C0186E8A80EB11CD5018C91882309F4B8
:102F30004AC0CCE0C81B8C3008F0C0E0F401EA5A6B
:102F4000FF4F81E080836401BEE4CB0ED11C60E0C2
:102F5000C6010E9412113401E3E56E0E711CD3010B
:102F60008C9103E0080FDDE24D2F481B4C0F83E0EE
:102F7000E82E24E560E0C6010E94651361E0C60109
:102F80000E941211F301808103E0080F4D2F481BAE
:102F90004C0F24E560E0C6010E940613F401E95AD3
:102FA000FF4F84E080833196D3018C91C81BC15DB3
:102FB000C083BC9660817181C6010E94A922F5017F
:102FC000808181508083DF91CF910F91EF90DF90CE
:102FD000CF90BF90AF909F908F907F906F9008950B
:102FE000CF92DF92FF920F931F93CF93DF93EC0169
:102FF0008C8D9D8D892B01F18E01025B1F4F40E06E
:1030000061E0C8010E941611FE01E95AFF4FDE017E
:10301000AE5ABF4F9C9185E5891B80833196108203
:10302000698D613009F46DC078F0888D653008F0E5
:1030300082C06B5F811175C0DF91CF911F910F919D
:10304000FF90DF90CF900895CE0185960E944A1F91
:1030500081E0FE01EA5AFF4F80836AEB73E0C8010A
:103060000E94C3151D8E1C8EFE01EC5AFF4F10826C
:1030700088EAF82E6E018AE0C80ED11CCE010E94AB
:10308000A0188823D9F369EA75E0C8010E94A92233
:103090006A8D7B8D4AE050E0C8010E94B82364E944
:1030A00075E0C8010E94A9226F2D62956F7070E0D3
:1030B0004AE050E0C8010E94A42369E875E0C80115
:1030C0000E94A92264E0C6010E9419108111B4CFA8
:1030D000FA94F110D3CF60E0CE010E94BD1F83B7F8
:1030E000817F846083BF83B7816083BF83B7816042
:1030F00083BF889583B78E7F83BF83B78E7F83BF5F
:10310000BDCFCF58DF4F88819981AA81BB818F7055
:103110009927AA27BB2767E00897A105B10508F002
:1031200068E7C801DF91CF911F910F91FF90DF9069
:10313000CF900C94D422882309F47ECF6FE2F1CF94
:103140008F929F92AF92BF92CF92DF92EF92FF92B7
:103150000F931F93CF93DF93EC017C0180E8E80E7F
:10316000F11CF70180809180A280B3800E94AC2086
:10317000861A970AA80AB90A6E01FFE7CF0ED11C7A
:10318000F601808190E0B0E0A0E08E0105581F4F6D
:1031900088159905AA05BB0508F04AC0F801808189
:1031A0009181A281B381892B8A2B8B2B09F440C09A
:1031B0000E94AC20F6012081620F711D811D911DBE
:1031C000F70160837183828393833F97808191812C
:1031D000A281B3810196A11DB11D80839183A28339
:1031E000B383F80110821182128213820E94B820E8
:1031F000FE01E958FF4F6083718382839383CE0180
:103200000E94C11FCE010A960E94EC0FCE01489683
:103210000E942A2081E0DF91CF911F910F91FF90B2
:10322000EF90DF90CF90BF90AF909F908F900895D8
:10323000F80180819181A281B381892B8A2B8B2B0C
:10324000A9F57E01F5E2EF0EF11CC7010E94051EF3
:10325000C7010E94781EC7010E943C1FCE010E9438
:103260008317CE010E94F0177E018EE4E80EF11C58
:10327000C7010E94CD10FE01EC5AFF4F80818111E1
:1032800003C0C7010E94B4100E94B820F8016083F7
:10329000718382839383FE01EB58FF4FC958DF4F40
:1032A00028813981621B730B7183608380E0B3CF07
:1032B0002F923F924F925F926F927F928F929F9246
:1032C000AF92BF92CF92DF92EF92FF920F931F9334
:1032D000CF93DF93CDB7DEB765970FB6F894DEBF17
:1032E0000FBECDBF6C016A8B7B8B4B83FC01EC5A0C
:1032F000FF4F10822FEF2D831C821D8A10E31C8A42
:103300003C013AE0630E711C842F90E09F838E8312
:103310002601E3E54E0E511C4601F5E28F0E911C8D
:103320009601295A3F4F39872887C601885A9F4FEF
:103330009B878A87F601EA5AFF4FFF87EE87225064
:103340003109398B288B0A971C01C6010E94A018ED
:103350008823D9F364E0C3010E941910012F110FD3
:10336000110B882399F0F201F081F1952B81F29FE6
:10337000202D112422502D8B64E0C3010E941910CE
:10338000811193C0C4010E94A51F94C065E0C301D0
:103390000E9419108111E7CF66E0C3010E94191045
:1033A0008111E1CF8C81811185C044E063E0C301CC
:1033B0000E942B10882331F09C899F5F9C8BC40155
:1033C0000E94A91F44E061E0C3010E942B108823E2
:1033D00031F0EC89E150EC8BC4010E94A91FFC89FB
:1033E0008F2F0F2E000C990B2E813F818217930790
:1033F00009F46BC0F7FF03C03B8131503C8BF201F5
:103400008081F4E0F80F2C89829FF0191124FD8B44
:103410009D89090F111D97FD1A9517FF02C00F5FB7
:103420001F4FF801F595E795FA83E9830981102F7D
:10343000E885F9851082EA85FB85008321E0EE8529
:10344000FF852083E889F9891082EA88FB88B12CFE
:10345000A12C2C89022E000C330B3D872C878E81EA
:103460009F818A159B0599F1EC85FD85EA15FB0581
:1034700079F423E0E885F9852083F2018081F02F3B
:103480002C89289FF00D11248F2FEA85FB858083DE
:10349000F70165917491C1010E94EF22FFEFAF1A0D
:1034A000BF0A22E0E20EF11CDACFC4010E94A11F84
:1034B0003C893D83C8013D89831B910937FD939564
:1034C000029764F181E08C83A3CF1C8A98CF60E0DF
:1034D000C1010E941211F20180814981FC89F89F8B
:1034E000400D1124415024E560E0C1010E943611D5
:1034F00061E0C1010E941211F201808103E0080F16
:103500004981FC898F9F400D1124425083E0E82EB1
:1035100024E560E0C1010E94061317CF8D816596F6
:103520000FB6F894DEBF0FBECDBFDF91CF911F91D4
:103530000F91FF90EF90DF90CF90BF90AF909F9052
:103540008F907F906F905F904F903F902F90089555
:103550000F931F93CF93DF93EC018C01025B1F4FFE
:10356000C8010E94B41061E675E0C8010E94A9225A
:10357000C8010E94CD1083E00E94232487E591E0DA
:10358000EEEFFFE30995FE01EC5AFF4F10826CE36A
:1035900075E0C8010E94EF22C8010E94CD102A9652
:1035A000CE010E94EC0F64E0CE010E94191081113F
:1035B00007C062E370E080E090E00E94DD20F0CF81
:1035C000DF91CF911F910F9108952F923F924F92CB
:1035D0005F926F927F928F929F92AF92BF92CF92A3
:1035E000DF92EF92FF920F931F93CF93DF93CDB7AC
:1035F000DEB729970FB6F894DEBF0FBECDBF99870F
:1036000088877B836A832A013C0180E7680E711CEE
:10361000F3018081882309F4F7C081E0E885F9850A
:10362000EA5AFF4F8083E885F985EB5AFF4F1082F5
:10363000E885F985EC5AFF4F1082E885F985108EF0
:103640008F01025B1F4F61E0C8010E941211888543
:1036500099858D5A9F4F9F838E83A884B98497E55F
:10366000A90EB11CE884F984E8E5EE0EF11C88840B
:103670009984F2E58F0E911C888599858F589F4F0C
:103680009D838C83288439849AE0290E311CC88458
:10369000D984E5E2CE0ED11C888599850E94A018B8
:1036A0008823D1F3EA81FB81F491F983FF2321F090
:1036B000EE81FF81F081F9832BEC35E040E060E0A2
:1036C000C8010E949C134114510439F04981445FA0
:1036D000920160E0C8010E949C13F50110828CE009
:1036E000F70180836A817B81C8010E94A922F401CD
:1036F0008081982F990F990F891B8D5AF50180832E
:10370000EE81FF818081982F990F990F891B835D2E
:10371000F7018083EC81FD81808167EC75E084FD99
:1037200002C063EC75E0C8010E94EF22F4018081C1
:10373000982F990F990F891B8D5AF5018083F701F6
:1037400080818F5F8083E885F98582A56FEB75E0C6
:10375000811102C06BEB75E0C8010E94EF22F401F9
:103760008081982F990F990F891B8D5AF5018083BD
:10377000F70180818F5F808367EB75E0C8010E944D
:10378000EF2265E0C1010E941910882351F0E885FD
:10379000F98562A56F5FC6010E94AD1FC6010E9438
:1037A000A91F64E0C1010E94191081111FC0F3011B
:1037B0002081422F50E070E060E0EC81FD8180814B
:1037C0009181A281B38184179507A607B70710F0EE
:1037D0002F3F61F466E0C1010E941910882309F4AB
:1037E0005BCF888599850E94A81A56CF8FEFF30189
:1037F000808360E0C6010E943F1FC6010E94A11F96
:1038000081E0E885F985808F29960FB6F894DEBFB0
:103810000FBECDBFDF91CF911F910F91FF90EF9021
:10382000DF90CF90BF90AF909F908F907F906F90E0
:103830005F904F903F902F90089550E040E00C949F
:10384000E51AE0E8F7E72591349181E02130304C2A
:1038500009F080E00895CF93DF93EC010E94211CD2
:103860009E01275A3F4FDE01A059BF4F882309F41C
:1038700040C0E6E9F7E78491F9018083E7E9F7E7DB
:10388000E491EC83E8E9F7E7E491ED83E9E9F7E710
:10389000859194919F838E83EBE9F7E785919491CD
:1038A00099878887EDE9F7E7E491EBA7EEE9F7E779
:1038B000E491EAA7EFE9F7E7E491EC93E0EAF7E7B0
:1038C000859194919D8F8C8FE2EAF7E78591949191
:1038D0009F8F8E8FE4EAF7E78591949199A388A34F
:1038E000E6EAF7E7859194919BA38AA3DF91CF91B4
:1038F00008958CE3F90180831C828FEF8D8320E291
:1039000033E03F832E8324ED33E03987288791E02D
:103910009BA79AA78C938CEA9DE09D8F8C8F8EED50
:103920009DE09F8F8E8F84E79EE099A388A38CE310
:103930009FE0DACFCF92DF92EF920F93CF93DF9396
:10394000EC01FC01E158FF4F82E38083349781E072
:1039500090E0A0E0B0E080839183A283B3833B97A3
:103960008FEF8083CE010E942B1CCE010E94B91FD5
:103970006FEFCE010E94BD1F6E018AE0C80ED11C00
:10398000C6010E94DC0FC6010E94EC0FCE014896D2
:103990000E9420208EE0E82E0FE020E14BE06DE059
:1039A000CE01825B9F4F0E94D715A596CE010E9443
:1039B0003E1D65E0C6010E941910882351F060E0A9
:1039C000CE01DF91CF910F91EF90DF90CF900C94CB
:1039D000AD1F40E06BE376E0CE01DF91CF910F9118
:1039E000EF90DF90CF900C94D21DCF93DF93D62F22
:1039F000C72F0E94211C882359F0AD2FBC2FEBE864
:103A0000F7E784918D933196E53987E7F807C9F791
:103A1000DF91CF910895CF93DF93DC0170E0660FC3
:103A2000771F1F96ED91FC915097E60FF71F259198
:103A3000349190963C932E935F97F9014591549160
:103A400014968C911497849F402D112491964C9339
:103A50009197F901C591D4916D2F70E04617170623
:103A600029F020F0F90125913491432F849F402DB6
:103A7000112492964C93DF91CF91089521E0FC019F
:103A8000248324E020A72AE936E0308B278760E0F2
:103A90000E940B1D61E070E083E00E945921E1EB80
:103AA000F0E08081887F81608083F89410928000AC
:103AB000E1E8F0E01082109285001092840088E125
:103AC00091E0909389008093880080818860808352
:103AD000808181608083EFE6F0E080818260808376
:103AE000789408950F93FC01011107C06230D9F05A
:103AF00030F4662379F0613091F00F9108956330CE
:103B0000C9F06430D1F76481649F402D1124458F42
:103B1000268FF3CF4B3008F04AE0468BEECF642F70
:103B20000F910C940B1D6481649F402D1124418FD3
:103B3000228FE3CF6481649F402D1124438F248F13
:103B4000DCCF80916D07882329F080916A078093EC
:103B5000B400089580E0FBCFFC01178A158A14A2F7
:103B600013A2108E10926A0710926B0710926D07C5
:103B70000C94A11D0F931F93CF93DF93EC018B0146
:103B80000E94AC1D1E870D871B8A1A8A81E08983DB
:103B900089E08E8B198E1B8E1D8EDF91CF911F9128
:103BA0000F910895411102C00C94BA1D0895CF934E
:103BB000DF93EC01611115C08881882391F0898120
:103BC00081110FC0E9858E2F90E0880F991FEF813A
:103BD000F885E80FF91F859194918F3F980721F49C
:103BE0001882DF91CF9108959C879927880F991F9C
:103BF000EA85FB85E80FF91F65917491CE010E945B
:103C0000BA1D89858F5F8987ECCF60E00C94D71D42
:103C10000F93CF93DF93EC01611166C089818823F4
:103C200009F462C08D8981115FC08D859E85EA8906
:103C3000FB89EE0FFF1FE80FF91F459154914115C5
:103C4000510541F42989213021F51B8A1A8AFC018A
:103C500045915491BA017695679576956795862F2B
:103C600040FF2EC0252F269526952695205186E0CB
:103C7000569547958A95E1F74F716F7000E0CE0138
:103C80000E94721DEA89FB893196FB8BEA8BCF017A
:103C90000AC019828881882369F060E0CE010E9401
:103CA000D71D8A899B89880F991FED85FE85E80FAE
:103CB000F91FCECFCE01DF91CF910F910C94AC1DA7
:103CC0008F738C8B8C81859F802D11248D8B1DA2F1
:103CD0001CA21BA281E08F8B80936D07188E8A89AE
:103CE0009B8901969B8B8A8BDF91CF910F910895D1
:103CF00060E00C94081ECF93DF93EC016111B3C018
:103D00008F89882309F4AFC08D89811105C0CE0148
:103D1000DF91CF910C94AC1D81508D8B8DA18111C1
:103D200034C02BA13CA12F5F3F4FC901880F991FC1
:103D3000EF8DF8A1E80FF91F85919491482F4770F6
:103D40004EA3492F469546954FA3AC0164E0569586
:103D500047956A95E1F74F739C81499F402D112447
:103D60004DA383FB882780F9809369073CA32BA38D
:103D700089A190E02817390740F02AA1222309F4ED
:103D800075C0821B91099CA38BA38DA181508DA32B
:103D9000888D31E0380F388F4C892FA1240F8C8506
:103DA000280F2A836B8D662361F070E0832F032E2A
:103DB000000C990B0E9462248C8D869F200D11248B
:103DC0002A838A8190E0CB966BE370E00E946224A4
:103DD0008A832E892B83698D662371F0062E000C51
:103DE000770B832F032E000C990B0E9462248A8D7F
:103DF000869F200D11242B836D8D662389F0832FE0
:103E0000330F990B70E00E946224CB0162E070E0F6
:103E10000E9462242E8D9B81289F900D11249B83EC
:103E20004F3341F18B818A300CF089E087FD80E0CF
:103E30008B83F894EA81F0E0E75BF94FE491E0933B
:103E40006C078D8198A5899F802D11249B81899F66
:103E5000802D11249EA1899F802D112480936B07B2
:103E600080936A077894DF91CF910895CE010E94E4
:103E7000AC1D8BCF1B82DDCF60E00C947B1ECF93FB
:103E8000DF93EC01611103C00E94AC1D1982DF9128
:103E9000CF910895CF93DF93EC010E94AC1D19825E
:103EA000DF91CF91089560916B07662329F180918E
:103EB0006E078F5F80936E0790916C078917E0F013
:103EC00081E090916D07911180E080936D071092D1
:103ED0006E0780916907882369F08091040193E45B
:103EE000899F802D1124895B809304010E944224C4
:103EF00090936A070C94A11D08951F920F920FB61C
:103F00000F9211242F933F934F935F936F937F935F
:103F10008F939F93AF93BF93EF93FF930E94531F91
:103F2000FF91EF91BF91AF919F918F917F916F9191
:103F30005F914F913F912F910F900FBE0F901F9067
:103F4000189562E976E00C94BA1D6AE876E00C9464
:103F5000BA1D64E876E00C94BA1DFC01862F660F4A
:103F6000990B668170E06F5F7F4F0E9462248583AA
:103F7000089521E0FC012083089570E085E00C9411
:103F80005921AF92BF92CF92DF92EF92FF920F939F
:103F90001F93CF93DF93EC0189819A812FE0289FB3
:103FA0008001299F100D112485E10E943E21800F80
:103FB000911F24E0969587952A95E1F79A83898346
:103FC0002881222391F1EC81AD80B12CD12CC12C20
:103FD000A885B9857D0110E000E06E817F819B019D
:103FE00050E040E08617970728F0BC01A817B907F2
:103FF00008F4BD0190E080E01F921F921F92EF93A2
:104000000E94BE236B830F900F900F900F9070E073
:1040100085E0DF91CF911F910F91FF90EF90DF909E
:10402000CF90BF90AF900C945921DF91CF911F9109
:104030000F91FF90EF90DF90CF90BF90AF900895D9
:10404000FC018CE39FE09383828384E0818381E0A1
:1040500084870895CF93DF93EC018C819D81892B18
:1040600021F18C858F7139F584E10E943E21BC01DC
:10407000990F880B990B0E94142526EE3FE34EEC16
:1040800050E40E94A0250E94E3249B017B836A8365
:10409000672BA9F084E08983FE01349680E041918A
:1040A00051912417350720F48983DF91CF9108952A
:1040B0008F5F8430A1F78C858F5F8C87F6CF8FEF71
:1040C0008983F9CF1F920F920FB60F9211242F936D
:1040D0003F938F939F93AF93BF938091700790917D
:1040E0007107A0917207B091730730916F0723E0B9
:1040F000230F2D3758F50196A11DB11D20936F0791
:104100008093700790937107A0937207B093730721
:104110008091740790917507A0917607B091770709
:104120000196A11DB11D8093740790937507A0930C
:104130007607B0937707BF91AF919F918F913F9191
:104140002F910F900FBE0F901F90189526E8230F08
:104150000296A11DB11DD2CF2FB7F89460917007C0
:104160007091710780917207909173072FBF089526
:104170003FB7F8948091740790917507A0917607E6
:10418000B091770726B5A89B05C02F3F19F001967F
:10419000A11DB11D3FBFBA2FA92F982F8827BC01A1
:1041A000CD01620F711D811D911D42E0660F771FC9
:1041B000881F991F4A95D1F70895CF92DF92EF9209
:1041C000FF92CF93DF936B017C010E94B820EB013B
:1041D000C114D104E104F10439F4DF91CF91FF90CF
:1041E000EF90DF90CF9008950E94B8206C1B7D0B5C
:1041F000683E734068F381E0C81AD108E108F1080D
:10420000C851DC4FE5CF789484B5826084BD84B515
:10421000816084BD85B5826085BD85B5816085BDC1
:10422000EEE6F0E0808181608083E1E8F0E01082DA
:10423000808182608083808181608083E0E8F0E01B
:10424000808181608083E1EBF0E080818460808305
:10425000E0EBF0E0808181608083EAE7F0E080813C
:10426000846080838081826080838081816080839C
:104270008081806880831092C10008958E3008F09C
:104280008E502091050190E4299F900111248770A0
:10429000822B80937C0080917A00806480937A00E6
:1042A00080917A0086FDFCCF809178009091790012
:1042B00008951F93CF93DF93182FEB0161E00E94C5
:1042C000DF21209739F460E0812FDF91CF911F919A
:1042D0000C941B22CF3FD10511F461E0F5CFE12F03
:1042E000F0E0EA55F94FE491E33031F140F4E13088
:1042F000B1F0E230E1F0C038D1057CF7E4CFE63030
:1043000029F1E73059F1E430B1F780918000806203
:1043100080938000D0938B00C0938A0004C084B542
:10432000806884BDC7BDDF91CF911F91089584B58A
:10433000806284BDC8BDF7CF809180008068809383
:104340008000D0938900C0938800EDCF8091B000A9
:1043500080688093B000C093B300E5CF8091B00037
:1043600080628093B000C093B400DDCF833081F0D1
:1043700028F4813099F08230A9F008958630A9F0B0
:104380008730C9F08430B1F4809180008F7D03C004
:10439000809180008F7780938000089584B58F7717
:1043A00084BD089584B58F7DFBCF8091B0008F7759
:1043B0008093B00008958091B0008F7DF9CFCF93A6
:1043C000DF9390E0FC01E654F94F24918253994F1A
:1043D000FC0184918823C9F090E0880F991FFC01AB
:1043E000EA50F94FA591B491FC01E451F94FC59100
:1043F000D49161110DC09FB7F8948C9120958223C0
:104400008C938881282328839FBFDF91CF910895C3
:10441000623051F49FB7F8943C91822F80958323AA
:104420008C93E8812E2BEFCF8FB7F894EC912E2B45
:104430002C938FBFEACF1F93CF93DF93162F282F94
:1044400030E0F901EA55F94F8491F901E654F94F4A
:10445000D491F901E253F94FC491CC23A1F0811119
:104460000E94B621EC2FF0E0EE0FFF1FE451F94F50
:10447000A591B4918FB7F894EC91111108C0D09523
:10448000DE23DC938FBFDF91CF911F910895DE2B48
:10449000F8CFCF93DF93282F30E0F901EA55F94F99
:1044A0008491F901E654F94FD491F901E253F94F9F
:1044B000C491CC23A1F081110E94B621EC2FF0E031
:1044C000EE0FFF1FEE51F94FA591B491EC91ED2342
:1044D00081E090E009F480E0DF91CF91089580E0E1
:1044E00090E0FACFCF92DF92EF92FF920F931F935B
:1044F000CF93DF936C01EB017B01E40EF51E10E01E
:1045000000E0CE15DF0561F06991D601ED91FC91D7
:104510000190F081E02DC6010995080F191FF1CF18
:10452000C801DF91CF911F910F91FF90EF90DF9025
:10453000CF900895FB0101900020E9F73197AF017A
:10454000461B570BDC01ED91FC910280F381E02DBD
:104550000994EF92FF920F931F93CF93DF937C0107
:104560008B01D0E0C0E0F80164910F5F1F4F66231C
:1045700059F0D701ED91FC910190F081E02DC70138
:104580000995C80FD91FEFCFCE01DF91CF911F91B1
:104590000F91FF90EF9008956115710511F00C9443
:1045A0009A2290E080E00895DC01ED91FC91019069
:1045B000F081E02D09940F931F93CF93DF93EC01CB
:1045C0006DE00E94D4228C016AE0CE010E94D422C8
:1045D000800F911FDF91CF911F910F9108950F933D
:1045E0001F93CF93DF93EC010E94A9228C01CE018F
:1045F0000E94DB22800F911FDF91CF911F910F91BD
:1046000008958F929F92AF92BF92CF92DF92EF92D6
:10461000FF920F931F93CF93DF93CDB7DEB7A19790
:104620000FB6F894DEBF0FBECDBF6C01142FE52F7F
:10463000CB01022F19A2223008F40AE07E0121E208
:10464000E20EF11C802E912CB12CA12C612F7E2F1B
:10465000A50194010E947624029F101911241A309A
:104660003CF5105DF70112937F01122FE32FCA0171
:10467000232B242B252B51F790E080E0E114F1044B
:1046800021F0B701C6010E949A22A1960FB6F894B4
:10469000DEBF0FBECDBFDF91CF911F910F91FF9075
:1046A000EF90DF90CF90BF90AF909F908F90089544
:1046B000195CD8CFCF92DF92EF92FF920F931F93A6
:1046C000CF93DF93EC016A017B012115310579F469
:1046D000E881F9810190F081E02D642FDF91CF9185
:1046E0001F910F91FF90EF90DF90CF9009942A30A7
:1046F0003105E9F42AE0F7FE1AC06DE20E94D422E7
:104700008C0144275527BA014C195D096E097F09B0
:104710002AE0CE010E940123800F911FDF91CF91EB
:104720001F910F91FF90EF90DF90CF900895B70108
:10473000A601CE01DF91CF911F910F91FF90EF90D5
:10474000DF90CF900C9401239A01AB01770F660B99
:10475000770B0C945A232115310541F4DC01ED91BE
:10476000FC910190F081E02D642F09940C940123B9
:104770009A01AB0170E060E00C94AB234F925F9222
:104780006F927F92AF92BF92CF92DF92EF92FF92A1
:104790000F931F93CF93DF93CDB7DEB729013A0173
:1047A0009B01AC01241935094609570989899A8961
:1047B000AB89BC89BC01CD016A197B098C099D09B3
:1047C0000E943224A8019701241935094609570986
:1047D0000E949824CA01B9016A0D7B1D8C1D9D1D84
:1047E000DF91CF911F910F91FF90EF90DF90CF90CD
:1047F000BF90AF907F906F905F904F90089561E071
:104800008AE00E941B2261E08AE00E94DF218CB5D1
:1048100080618CBD8CB580648CBD61E08DE00E94B0
:10482000DF2161E08BE00C94DF21811104C08CB5A5
:1048300080628CBD08958CB58F7DFBCF9CB5937F36
:10484000892B8CBD08959CB59C7F282F2370922BBB
:104850009CBD9DB582FB222720F9892F8E7F822B5C
:104860008DBD0895DB018F939F930E94B724BF9164
:10487000AF91A29F800D911DA39F900DB29F900DAF
:1048800011240895991B79E004C0991F961708F028
:10489000961B881F7A95C9F780950895AA1BBB1BA4
:1048A00051E107C0AA1FBB1FA617B70710F0A61B30
:1048B000B70B881F991F5A95A9F780959095BC0151
:1048C000CD01089597FB072E16F4009407D077FDCD
:1048D00009D00E944E2407FC05D03EF490958195A6
:1048E0009F4F0895709561957F4F0895A1E21A2E0C
:1048F000AA1BBB1BFD010DC0AA1FBB1FEE1FFF1F84
:10490000A217B307E407F50720F0A21BB30BE40BD3
:10491000F50B661F771F881F991F1A9469F760951A
:104920007095809590959B01AC01BD01CF010895D4
:10493000052E97FB1EF400940E94AF2457FD07D06C
:104940000E94762407FC03D04EF40C94AF245095BB
:104950004095309521953F4F4F4F5F4F089590956B
:104960008095709561957F4F8F4F9F4F08950E945E
:10497000D424A59F900DB49F900DA49F800D911DF0
:10498000112408950024A7FD00942A0F301D401D16
:10499000501D601D701D801D901D0895EE0FFF1F9E
:1049A0000590F491E02D0994A29FB001B39FC0013E
:1049B000A39F700D811D1124911DB29F700D811D4B
:1049C0001124911D08950E947F2588F09F5798F02B
:1049D000B92F9927B751B0F0E1F0660F771F881F04
:1049E000991F1AF0BA95C9F714C0B13091F00E941E
:1049F0009925B1E008950C949925672F782F882781
:104A0000B85F39F0B93FCCF3869577956795B39544
:104A1000D9F73EF490958095709561957F4F8F4FB3
:104A20009F4F0895E89409C097FB3EF490958095B8
:104A3000709561957F4F8F4F9F4F9923A9F0F92F64
:104A400096E9BB279395F695879577956795B795E2
:104A5000F111F8CFFAF4BB0F11F460FF1BC06F5FC8
:104A60007F4F8F4F9F4F16C0882311F096E911C0DA
:104A7000772321F09EE8872F762F05C0662371F0FB
:104A800096E8862F70E060E02AF09A95660F771F0F
:104A9000881FDAF7880F9695879597F9089597F903
:104AA0009F6780E870E060E008959FEF80EC0895D4
:104AB00000240A94161617061806090608950024FD
:104AC0000A9412161306140605060895092E039477
:104AD000000C11F4882352F0BB0F40F4BF2B11F4EB
:104AE00060FF04C06F5F7F4F8F4F9F4F089557FD4A
:104AF0009058440F551F59F05F3F71F04795880F4C
:104B000097FB991F61F09F3F79F0879508951216E2
:104B100013061406551FF2CF4695F1DF08C016168E
:104B200017061806991FF1CF86957105610508943F
:104B30000895E894BB2766277727CB0197F9089556
:104B40000E94B3250C9466250E94582538F00E94D7
:104B50005F2520F0952311F00C944F250C945525DA
:104B600011240C949A250E94772570F3959FC1F328
:104B7000950F50E0551F629FF001729FBB27F00D0B
:104B8000B11D639FAA27F00DB11DAA1F649F662760
:104B9000B00DA11D661F829F2227B00DA11D621FAF
:104BA000739FB00DA11D621F839FA00D611D221F69
:104BB000749F3327A00D611D231F849F600D211D4D
:104BC000822F762F6A2F11249F5750409AF0F1F0D0
:104BD00088234AF0EE0FFF1FBB1F661F771F881F39
:104BE00091505040A9F79E3F510580F00C944F25FD
:104BF0000C949A255F3FE4F3983ED4F3869577951D
:104C00006795B795F795E7959F5FC1F7FE2B880FDE
:104C1000911D9695879597F908958F929F92AF92DF
:104C2000BF92CF92DF92EF92FF92CF93DF93EC018E
:104C3000688179818A819B81611571058105910562
:104C400021F464E279ED8BE597E02DE133EF41E06B
:104C500050E00E94982449015A019B01AC01A7EA47
:104C6000B1E40E94B7246B017C01ACEEB4EFA50166
:104C700094010E942129DC01CB018C0D9D1DAE1DEC
:104C8000BF1DB7FF03C00197A109B048888399836E
:104C9000AA83BB839F77DF91CF91FF90EF90DF9046
:104CA000CF90BF90AF909F908F9008950E940D2657
:104CB000089580E091E00E940D260895B0E0A0E004
:104CC0008093000190930101A0930201B09303012E
:104CD0000895DC0101C06D9341505040E0F7089504
:104CE000AEE0B0E0E6E7F6E20C9434290D891E89C7
:104CF0008F89988D26E02C831A83098397FF02C041
:104D000080E090E801979E838D83AE01455E5F4F02
:104D1000698D7A8DCE0101960E94A0264D815E811B
:104D200057FD0AC02F813885421753070CF49A01AA
:104D3000020F131FF80110822E96E4E00C94502904
:104D4000ABE0B0E0E6EAF6E20C9426297C013B01F8
:104D50008A01FC0117821682838181FFC8C1CE01BE
:104D600001965C01F7019381F30193FD859193FF17
:104D700081913F01882309F453C1853239F493FDB1
:104D8000859193FF81913F01853229F4B70190E02D
:104D90000E949028E7CF912C212C312CFFE1F315B4
:104DA00038F08B3211F190F4803209F1833229F11D
:104DB00037FC3CC020ED280F2A3050F536FE20C0CD
:104DC0008AE0989E200D1124922E06C08D3291F01B
:104DD000803371F7689430F8F30193FD859193FF68
:104DE00081913F018111DACF21C0689431F8689434
:104DF00032F8F2CF689433F8EFCF689434F8ECCF00
:104E0000EAE02E9E200D1124222E689435F8E4CF7E
:104E10008E3229F436FC04C1689436F8DDCF8C3626
:104E200019F4689437F8D8CF8836B1F2982F9F7D5F
:104E300095549330E0F08336A1F18337C1F1833587
:104E400009F063C02801F2E04F0E511CF801C08048
:104E5000D180692D70E036FC02C06FEF7FEFC60194
:104E60000E947A284C01689437F882010AC00C5FCE
:104E70001F4FFFE3F98388248394912C6501E89404
:104E800037F833FE2DC0522C8114910471F5552052
:104E900009F468CFB70180E290E00E9490285A940C
:104EA000F6CFF801808189830E5F1F4FE4CF280180
:104EB000F2E04F0E511CF801C080D180692D70E0E6
:104EC00036FC02C06FEF7FEFC6010E9485284C01BF
:104ED0008201D5CFB70180E290E00E9490282A9409
:104EE0002814190409F0B0F7CECFF60137FC8591EC
:104EF00037FE81916F01B70190E00E949028511018
:104F00005A94F1E08F1A9108BFCF843619F0893690
:104F100009F077C0F80137FE6BC060817181828132
:104F200093810C5F1F4FF32DFF763F2E97FF09C033
:104F300090958095709561957F4F8F4F9F4F6894A6
:104F400037F82AE030E0A5010E94C028C82ECA1810
:104F50008C2C432C36FE0CC0E89440F8C91440F465
:104F600034FE05C032FC03C0F32DFE7E4F2E892C8B
:104F700044FE95C0FE01EC0DF11D8081803309F0E7
:104F800087C0242D297E422E842D8870582E43FC04
:104F900095C040FE8FC09C2C821418F42C0C922CCF
:104FA000981844FE91C0B70180E390E00E949028D9
:104FB00042FE09C088E790E041FE02C088E590E02B
:104FC000B7010E949028C91408F48AC0CA94D12C51
:104FD0009FEFC91AD90ACA0CDB1CF60182916F0136
:104FE000B70190E00E949028AC14BD04B1F74FCFF8
:104FF00060817181072E000C880B990B0E5F1F4F8B
:1050000092CFD32CE894D4F82AE030E0853739F1F8
:10501000232D297FD22E8F3601F148F48835A9F04F
:10502000F701868197812B96E2E10C944229803723
:1050300049F08837A9F7D4FE02C06894D2F820E17D
:1050400030E00DC06894D4F8F6CF34FE03C0822F50
:105050008660D82E20E132E002C028E030E0F8017E
:10506000D7FE0FC060817181828193810C5F1F4FD9
:10507000A5010E94C028C82ECA183D2CE89437F814
:1050800067CF6081718190E080E00E5F1F4FF0CFAD
:1050900042FC02C0839478CF8394839475CF842D8F
:1050A000867809F471CFF6CFB70180E290E00E94D4
:1050B000902883948214C0F3512C73CF522C58182B
:1050C000821408F46ECFF8CF842D867809F47BCF54
:1050D0008BE241FE80E247FC8DE2B70190E071CFA8
:1050E000B70180E390E00E9490289A946CCF8FEFF4
:1050F0009FEF99CFFC010590615070400110D8F7E7
:10510000809590958E0F9F1F0895FC01615070400F
:1051100001900110D8F7809590958E0F9F1F0895EC
:105120000F931F93CF93DF93182F092FEB018B81E0
:1051300081FD09C01FEF0FEF812F902FDF91CF91DD
:105140001F910F91089582FF14C02E813F818C81A1
:105150009D81281739073CF4E881F981CF01019638
:105160009983888310838E819F8101969F838E838C
:10517000E3CFE885F985812F0995892BA1F3DACF53
:10518000FA01AA27283051F1203181F1E8946F9378
:105190006E7F6E5F7F4F8F4F9F4FAF4FB1E03ED01E
:1051A000B4E03CD0670F781F891F9A1FA11D680FBC
:1051B000791F8A1F911DA11D6A0F711D811D911DEF
:1051C000A11D20D009F468943F912AE0269F112464
:1051D0003019305D3193DEF6CF010895462F4770C8
:1051E000405D4193B3E00FD0C9F7F6CF462F4F7023
:1051F000405D4A3318F0495D31FD4052419302D081
:10520000A9F7EACFB4E0A695979587957795679526
:10521000BA95C9F700976105710508959B01AC0126
:105220000A2E06945795479537952795BA95C9F74D
:10523000620F731F841F951FA01D0895B7FF0C9464
:10524000B7240E94B724821B930B08952F923F929C
:105250004F925F926F927F928F929F92AF92BF9286
:10526000CF92DF92EF92FF920F931F93CF93DF9332
:10527000CDB7DEB7CA1BDB0B0FB6F894DEBF0FBE8F
:10528000CDBF09942A88398848885F846E847D84DC
:105290008C849B84AA84B984C884DF80EE80FD80DE
:1052A0000C811B81AA81B981CE0FD11D0FB6F89454
:1052B000DEBF0FBECDBFED01089513E0C2E8D3E01D
:1052C00004C0FE010E94CE242196C338D107C9F73D
:0452D000F894FFCF80
:1052D40001000000010148503D257500573D25643B
:1052E40000473D256400463D256400FA000000FDAA
:1052F40000030004000400422E4241525200415473
:105304005441434B00432E504541532E0027012E58
:1053140001350101000000000019006400C800000C
:0E532400000000451772224C4F4144455200D4
:040000030000075A98
:00000001FF
